:10000000AD0B060C2500F609320C960003071D0AFD
:100010001D023500020C950096000307170A1D0209
:100020003500020CD501960003071B0A1D0A87053F
:10003000A704D405200AA705200AD4048704A7042E
:10004000050C2500F609320C960003073C0A1C0239
:100050003500050C950096000307360A1C02350092
:10006000050CD501960003073C0A390AF105D104B5
:100070003E0AD105F1043E0AF104D104020C250028
:10008000F609320C96000307540A820C9600030707
:10009000540AAA0C960003074E0A510AE705C70442
:1000A000560AC705E705560AE704C704030C2500EE
:1000B000F609320C960003076C0A820C96000307BF
:1000C0006E0AAA0C96000307690A660A67055B04B4
:1000D000770A5B046704770A6704770A5B06770A86
:1000E000A607750AA6045B05770AA6055B05040C3E
:1000F0002500F609320C960003079D0A820C960033
:100100000307870AAA0C960003079B0A910A1B069D
:100110009D0A91078E0A91041B059D0A91051B05F6
:100120009D0A3B069D0AB107980AB1043B059D0A4A
:10013000B1053B059D0A1B043B046500F609320C22
:1001400096000307CB0A900C96000307AC0AA00C9C
:1001500096000307CA0ABB0A7B06CB0A960C350039
:100160001F0295009E004307B70A7B05CB0A1F02BA
:10017000BE007B05CB0A7B06CB0A960C35001F021E
:10018000D5019E004307C60A7B05CB0A1F02FE016C
:100190007B05CB0A7B04010C2500F609320C960086
:1001A0000307010A820C96000307EE0AAA0C9600C8
:1001B0000307E00AC30C0607690C3800F405010ABE
:1001C000F407E50A960C3800F404D406B407010AD3
:1001D000730C0607B90C3800B404010AD407010AED
:1001E000AF0C06077D0C3800B405010A72007300DD
:1001F00079007700140434040000000000000000BF
:1002000000000000000000000000000000000000EE
:10021000000000000000000000000000B9024306DA
:10022000B702B2024306B30200006507230B1407AE
:10023000320B340514041202390013023700720025
:1002400073000000FC0A00001405090C0000000007
:100250000000930003063B0B3407FC0A340412022F
:100260003600400B090C0000930003063D0B000014
:1002700000000000FC0A7600400BFF0C3600400B2B
:10028000B9024306B7020A0C3200F202450B000025
:10029000090C97000307400B720012029E0007052D
:1002A0004307540B07045A0B0A0C3300F302560B96
:1002B000B2024D0B72001202980066054307620BF2
:1002C0006604680B0A0C3300F302640BB2025B0B8A
:1002D000B002150C90000307740B70007407720BCA
:1002E0007404740B7405740BBA02080C9A000307AB
:1002F000800B7A0094077E0B9404800B9405800B8E
:10030000B107870B7407870BC605E6059B0BE60450
:10031000C604B1069B0BF107910B7407910BE60520
:100320009B0BE604B1069B0BD1079A0B74079A0B43
:10033000C6059B0BC6049107A90B94070008270666
:10034000A50B2705470494040008270447059404D7
:1003500000082704470494040008960C3E00380067
:10036000080C0500010C0600000C07007100660077
:100370006700070C0200350C300061000000FE0C25
:1003800081000307BE0BF002BD0B060C2500F60929
:1003900016023D00050C2500F60916023C00460534
:1003A000500C9D0003074604500C9C0003074604B4
:1003B0002605010C0600200C3300FF0C3200F2026F
:1003C000DF0BF302DD0B0B0C060026047200240C7D
:1003D00033002607F60B010C0600030C0600F3029F
:1003E000E90BB202FA0C92000307E70B12023F007E
:0203F000010A00
:0203FE00000AF3
:080400000F000F000F000F00B8
:021FFE00FA0FD8
:00000001FF
